:020000040000FA
:10000000831670308F001528C0000408C100030853
:10001000C2000A08C300EF2043088A004208830098
:1000200041088400C00E400E090003309B004030A0
:100030009F0023308500D73081000C3086002430AB
:10004000980019309900831240309F00903098003A
:10005000FF308500FF308600203084008001840A54
:1000600044300402031D2E280F30861DB9000130D4
:10007000AB00FF30BB00BC00BD003B30BE00E73032
:100080008100A0308B008C1E43281819AB289818CB
:10009000AB281A08A0004C3C031D5128A9172913AE
:1000A00057282008523C031D99282917A9138C1E94
:1000B00057281819AB289818AB281A080F39A00030
:1000C0000310200DA000A00DA00D2007AA008C1E7B
:1000D00067281819AB289818AB281A080F39AA07EF
:1000E0008C1E70281819AB289818AB281A08A00085
:1000F0004D3C031D872806308722A912291601309E
:10010000AB00AD01AE01AF01FE30BD0043282008B9
:10011000483C031DA828063087222912A916013061
:10012000AB00AD01AE01AF01FE30BD003B30BE0003
:1001300043282008543C031DA2282908A8000F3991
:10014000A900B1282008533C031D4328063087220C
:100150000F30A90543281A08181218160F30A905E0
:100160004328AF1BB128AC015D22A600A7010A30CD
:100170002602031CBE28A600A70AB7284C308722F7
:100180002708303E87222608303E87224830A81EA6
:100190004D3087220D3087220A3087225D22A6004B
:1001A0005D22A700263049225D22A7002730352294
:1001B000AE0BCE280630872243280F398207A034A1
:1001C000F93464347034393432342234F83420341D
:1001D00038347F3423346734613426342E340B1D95
:1001E0000800E73081000B11FF308600FF308500EA
:1001F000BB0A3B080339031D0129EF30291885008C
:100200002929A91C29298619092929193B1F0D29E2
:100210002929A91D0D293B1B2929A100A103323041
:1002200086193630210784000008DD208500A100F2
:10023000A11C8610211C06103B080339A100A10354
:10024000031D242986132929A10B282906132929EE
:100250000612AF1F5B29831603178C185B290C113C
:10026000831203132C0884000008831203178C00E8
:10027000831203132D08831203178D0083160317AF
:100280008C130C1555308D00AA308D008C14831200
:100290000313AD0A01302F1B0430AC072F172C08B5
:1002A000393C031D5B29AF13AE0A2E08553C031DD4
:1002B0005B290F30A905831203133B087F39031D07
:1002C0009129712230308400B1212911A31B2915F5
:1002D0000F302305B2002408B3002508B4003530E0
:1002E0008400F221A911A31BA9150F302305B60024
:1002F0002408B7002508B800B90E0F30B904F03053
:10030000861DB905390E390603198929A9149430B7
:10031000BA00BA0B8D29BA0AA9102908C039031DE1
:100320002910BC0F08000730BC002908C039013073
:100330000319A906BD0F0800B530BD00291AAB0B83
:10034000A4292A08AB000922BE0A3C303E02031D44
:100350000800BE01A91AAB0B08002A08AB0009224D
:100360000800A301A5010008A200840A0008E63CD9
:10037000A4000318D029FF3A013EA400093C031C45
:10038000CC296430A407A2080319EB29A20E03109C
:10039000220C013EA500EB29A3176430A400EB2931
:1003A000633C031CE029A2080319EB29A4080319E4
:1003B000C129A20E0310220C093CA500A403EB29BD
:1003C0002408643C031DA2016430A400A208031D9C
:1003D000D929A317A4010A302402031C0800A40091
:1003E000A30AEB29A301C8300002031CFB29A317B1
:1003F000A401A50108000310000CA400003003189C
:100400000530A5000A302402031C0800A400A30A3A
:10041000022AA91F2F2A831603170C118312031314
:100420002D08831203178D00831203132A082F1B34
:100430003008831203178C00831603178C130C15D6
:1004400055308D00AA308D008C1483120313AF1722
:10045000AD0A30302F1B3130AC0029140800291FA1
:10046000080029143030492235308400F221483008
:1004700087222308303E87222408303E87222E30F0
:1004800087222508303E87220D3087220A308722B6
:1004900008008400B121543087222308303E87228F
:1004A0002408303E87222E3087222508303E8722BE
:1004B0000D3087220A3087220800831603170C119B
:1004C000831203132C08831203178D00831603175E
:1004D0008C130C14831203170C0883120313AC0A39
:1004E000080041309F008F221F151F19752A1E0812
:1004F000B10083161E088312C039B00049309F0036
:100500008F221F151F19822A1E08B50008008B13A1
:100510008316981C892A831299008B1708000830CB
:0E052000BF000000BF0B912A00000000080081
:02400E00303F41
:02401000FC3F73
:00000001FF
